:100000007A28A60001300428A10027082502031D34
:100010000B2826082402043003180130031902308B
:100020002105031D01307528A000240825040319AB
:1000300075286F20A701A801200984178005841363
:10004000000022282608A70700082004031C200619
:100050008000A80A0319A40A0319A50F2028200864
:1000600084178004752883169B0083161C141A08B5
:100070009B0A752883169A001C1555309D00AA30DE
:100080009D009C149C1842281C119B0A7528800115
:10009000840AFF3E031D47287528A701A600FF30EC
:1000A000A607031CA707031C75280330A500DF3033
:1000B0005B204F28A501E83EA400A509FC30031CE5
:1000C0006428A40703186128A4070000A50F61286D
:1000D00024186A28A41C6E2800006E280800A409B1
:1000E000A509A40A0319A50A0800831383120313A0
:1000F0000000080007309900CC3083168500811776
:1001000083128501203084004030472003303320A3
:10011000B700AD1602303320B8001330B10088307C
:10012000B000CC28AD13851D9628AD178519AD14E8
:10013000851DAD10BA0103018519013EAD18013CC2
:1001400003190130031D0301AC0032303A020130C3
:10015000031803012C050319AF28BA0A9B280330A2
:10016000A500E8305B200800370838020318B928DA
:10017000B80A380837020318BE28B8033808A600A2
:10018000A5010230A4000530840004301420380892
:100190003702031DB4280800051285100510310828
:1001A0003004031DE4283808A600A5010230A4008D
:1001B00005308400043014201330B1008830B000C2
:1001C000AD1EE428AD12B420B003300A0319B10308
:1001D0008519CF2850304D2005162730AF0010303C
:1001E000AE00030185190130AC002F08A5002E08D0
:1001F000A400A701013001202C0503190429AE0336
:100200002E0A0319AF03F1282F082E04031D092914
:10021000CC28BA01013085190301AC0034303A0210
:100220000130031803012C0503191829BA0A0A29F9
:1002300034303A0203181D29CC280130A500F430CF
:100240005B2092200301AD1B0130013A03193613E4
:10025000031D361792202D17AD1F2D13922039162E
:10026000AD1F39129220B915AD1FB9119220391561
:10027000AD1F39119220B914AD1FB9109220391455
:10028000AD1F39109220B616AD1FB6129220361649
:10029000AD1F36129220B615AD1FB611922036153D
:1002A000AD1F36119220B614AD1FB6109220361431
:1002B000AD1F3610AD1E9E2905143608031D622998
:1002C0006430B60001303602031D7129B6012D14C9
:1002D0002D1502303320B80083169B018312390894
:1002E0003A200D303602031D7F29013083169B0012
:1002F000FF3083123A2078303A20B4303A20203050
:100300003602031D8E29B6012D14AD15023033209F
:10031000B80083169B01831239083A202130360237
:10032000031D9D29B6012D102D1601303320B80074
:1003300083169B01831239083A20B6290301332022
:10034000A2003908220203190130031D0301AC0089
:100350000130360203190130031D03012C05031976
:10036000B629851403303320B700B42003013320AD
:10037000A2003908220203190130031D0301AC0059
:100380002030360203190130031D03012C05031927
:10039000CB292D14B60103013320A2003908220213
:1003A00003190130031D0301AC002130360203198B
:1003B0000130031D03012C050319E0292D10B6019E
:1003C0003608031D672A03013320A20039082202E0
:1003D00003190130031D0301AC0039080319013072
:1003E000031D03012C040319672AAD1AF82985148B
:1003F0002D1C0D2AAD1D022AFF3038020318012AD8
:10040000B80A0C2A01303320A2002208380203184F
:100410000B2AB80A0C2A85101E2A2D1E142AB80889
:100420000319132AB8031E2A02303320A200380809
:10043000220203181D2AB8031E2A85103808A600B8
:10044000A5010230A40005308400043014200130DE
:10045000B3002C30B2003308B5003208B400B20843
:10046000031D352AB3080319462AB203320A0319B9
:10047000B303851D402AB403340A0319B503412A86
:10048000462A0130A500F4305B202F2A1430AD1E1F
:100490000301AA000301AD1E0301AB0005302A07CA
:1004A000A6002B080318013EA70026084E20350899
:1004B0003302031DF82934083202031DF829030111
:1004C0002D180130013A03192D10031D2D14AD1EF6
:1004D000BB2AAD122D1D732A033083169B00831295
:1004E00038083A20A62AAD1D8C2A013083169B00BD
:1004F000831238083A2003303320A2000130332021
:10050000A3002208230203188B2A033083169B00C2
:10051000831238083A20A62A2D1EA52A02308316F7
:100520009B00831238083A2003303320A2000230A7
:100530003320A300230822020318A42A03308316C1
:100540009B00831238083A20A62ACC28BA01013031
:1005500085068316051002308312850683168510E2
:10056000963083124D20BA0A0F303A02031DA72A93
:0C0570002D11AD112D1264304D20CC284F
:02400E00843FED
:084200000000FF007800B4008B
:00000001FF
